:1000000013C0189518951895189518951895189562
:10001000189518951895F2C3189518951895189570
:1000200018951895189518958FE181BD87E181BDC8
:100030008FE58DBFC0E4E8E34E2E84E08EBFD4E0B0
:10004000F4E05F2EEEEFF3E0A0E6B0E088278D93BA
:100050003197E9F78CE089B988E18AB940D3662401
:1000600080EC81BB8FE084BB81E087BB81E0809323
:10007000840081E08093830032D321D38FE914E0A0
:100080002CD3E4EDF8E015D3579A579A7894CDD253
:10009000082F003009F4FBCFD2D2A0E6B0E08D9358
:1000A00088278C9302D09FD0F2CFA0E6B0E0E0EE9C
:1000B000F8E0FDD309F005C0709185007068709379
:1000C00085000027A5E8B0E08C9187FB0EF401E0E5
:1000D00041E0041709F086C0E0E6F0E0A3E6B0E0F6
:1000E0009DD2DAD3A3E6B0E0DCD3082F033010F0C2
:1000F00009F001C009C0A3E6B0E088278C93709195
:1001000085007F7770938500A3E6B0E0E2EEF8E02B
:10011000CED309F031C084E690E027D3E6EEF8E0D4
:10012000B3D2B8D2E8EEF8E0AFD2B4D2A3E6B0E0F2
:1001300088278C93709185007F77709385007091EC
:1001400085007F7B70938500709185007F7D709323
:10015000850081E080938600AEE6B0E088278C932E
:1001600081E08093840081E080938300A8E6B0E082
:1001700088278C93C09836C0ECEEF8E098D309F04D
:1001800031C084E690E0F1D2E6EEF8E07DD282D292
:10019000E0EFF8E079D2A3E6B0E088278C93709185
:1001A00085007F77709385007091850070647093EF
:1001B00085008FE711E091D2E4EFF8E07AD28FE981
:1001C00011E08BD2E4EFF8E074D28FEB11E085D22E
:1001D000E4EFF8E06ED28FED11E07FD2E4EFF8E0CB
:1001E00068D2C09A08950027A5E8B0E08C9186FBFC
:1001F0000EF401E041E0041709F015C0A0E6B0E0FC
:1002000034D3ABE6B0E00C9300916B000A3E09F0EA
:100210000AC0709185007F7B709385007091850086
:100220007F7D709385000027A5E8B0E08C9186FB68
:100230000EF401E041E0041709F012C0E0E6F0E03E
:10024000A8E6B0E0EBD128D3A8E6B0E02AD3082F87
:10025000023009F005C0A6E8B0E08C918F5F8C9366
:100260000027A5E8B0E08C9185FB0EF401E041E0A9
:10027000041709F0C5C0A8E6B0E013D3082F023078
:1002800009F0BEC0A8E6B0E0EAE0F9E010D309F05A
:100290000DC0AEE6B0E088278C93A4E8B0E08C9166
:1002A0008F5F8C9381E080938300AAC0BFD0ECE67F
:1002B000F0E0AEE6B0E0B2D1EFD2009184000130C0
:1002C00009F04CC0AEE6B0E0ECD2082F053009F0E2
:1002D00006C0AEE6B0E0A2D1EEE0F9E099D1AEE61C
:1002E000B0E0E4E1F9E02FEF91E053D2002F0030CD
:1002F00010F009F001C00FC0AEE6B0E088278C9383
:100300008FE711E0EAD1E8E1F9E0D3D1AEE6B0E061
:10031000EEE2F9E07DD1AEE6B0E0EAE3F9E02FEFFE
:1003200091E037D2002F003010F009F001C00FC06B
:10033000AEE6B0E088278C938FE711E0CED1E8E1FC
:10034000F9E0B7D1AEE6B0E0E2E4F9E061D18FE7E1
:1003500011E0C3D1AEE6B0E0A6D152C0023009F040
:100360002CC000918300023009F004C0AEE6B0E07A
:1003700088278C93AEE6B0E0E0E5F9E02FEF91E05E
:1003800008D2002F003010F009F001C00FC0AEE617
:10039000B0E088278C938FE911E09FD1E8E1F9E084
:1003A00088D1AEE6B0E0E4E5F9E032D18FE911E0C2
:1003B00094D1AEE6B0E077D123C0033009F017C086
:1003C0008FEB11E08AD1AEE6B0E06DD1AEE6B0E0E1
:1003D00068D2082F043109F009C0A4E8B0E08C917C
:1003E0008F5F8C93AEE6B0E088278C9309C0043011
:1003F00009F006C08FED11E070D1AEE6B0E053D148
:1004000000918600053109F005C070918500706289
:1004100070938500A8E6B0E044D2082F023009F0BE
:1004200004C0A8E6B0E088278C930895A8E6B0E061
:10043000ECE5F9E03CD209F006C0ACE6B0E0E0E65D
:10044000F9E0E6D0DFC0E2E6F9E031D209F006C01B
:10045000ACE6B0E0E6E6F9E0DBD0D4C0E8E6F9E0EF
:1004600026D209F006C0ACE6B0E0ECE6F9E0D0D068
:10047000C9C0EEE6F9E01BD209F006C0ACE6B0E078
:10048000E2E7F9E0C5D0BEC0E4E7F9E010D209F038
:1004900006C0ACE6B0E0E8E7F9E0BAD0B3C0EAE7FE
:1004A000F9E005D209F006C0ACE6B0E0EEE7F9E00D
:1004B000AFD0A8C0E0E8F9E0FAD109F006C0ACE698
:1004C000B0E0E4E8F9E0A4D09DC0E6E8F9E0EFD1BF
:1004D00009F006C0ACE6B0E0EAE8F9E099D092C0D5
:1004E000ECE8F9E0E4D109F006C0ACE6B0E0E0E900
:1004F000F9E08ED087C0E2E9F9E0D9D109F006C071
:10050000ACE6B0E0E6E9F9E083D07CC0E8E9F9E0E8
:10051000CED109F006C0ACE6B0E0ECE9F9E078D065
:1005200071C0EEE9F9E0C3D109F006C0ACE6B0E075
:10053000E2EAF9E06DD066C0E4EAF9E0B8D109F08A
:1005400006C0ACE6B0E0E8EAF9E062D05BC0EAEAF7
:10055000F9E0ADD109F006C0ACE6B0E0EEEAF9E0B2
:1005600057D050C0E0EBF9E0A2D109F006C0ACE6EC
:10057000B0E0E4EBF9E04CD045C0E6EBF9E097D110
:1005800009F006C0ACE6B0E0EAEBF9E041D03AC0D1
:10059000ECEBF9E08CD109F006C0ACE6B0E0E0ECA1
:1005A000F9E036D02FC0E2ECF9E081D109F006C0C5
:1005B000ACE6B0E0E6ECF9E02BD024C0E8ECF9E0E2
:1005C00076D109F006C0ACE6B0E0ECECF9E020D062
:1005D00019C0EEECF9E06BD109F006C0ACE6B0E072
:1005E000E2EDF9E015D00EC0A8E6B0E03ED1ABE6F2
:1005F000B0E00C93ABE6B0E08C91ACE6B0E08D934C
:1006000088278C93A3E8B0E08C918F5F8C9308953A
:10061000C8950D9231960020D9F708958F938D914A
:100620008823E9F711978F9108958091B9009091EF
:10063000BA00891711F081E00895882708959F93E3
:100640008091B9009091BA0089179F9111F4882781
:1006500008950F929F93AF93BF938091B9009091AB
:10066000BA008917D1F3A7E8B0E0A90F0024B01DA4
:100670008C919395923309F499279093BA00BF9186
:10068000AF919F910F900895AFD0802D11F005D0BC
:10069000FBCF08958DE001D08AE05D9BFECF8CB941
:1006A0000895A8E2B4E08D91882311F02CD0FBCFFF
:1006B00008959AD0802D11F026D0FBCF089581E0C7
:1006C00024D041D008958FE7213039F08FE92230CE
:1006D00021F08FEB233009F08FED810F16C033D05E
:1006E00032D031D030D0A09AA19AA29AA39A8E9AF1
:1006F0008F9A84E20AD089E008D080E206D086E0B2
:1007000004D08CE002D0979A01C0979828E0C1707D
:100710008795661F6C2B2A95D1F7862F8295682FB7
:1007200082958F7053B3507F852B85BB06D06F7039
:10073000652B65BB02D00CD00895969A000000008E
:100740000000969808958FEF03D08A95E9F70895F1
:1007500065EA6A95F1F708953197F1F7089568947D
:1007600062F80895E89462F80895EF93FF93EE27F6
:10077000E82BE92B31F0E8EEF3E03197F1F7019740
:10078000D1F7FF91EF91089599910027A90FB01F1C
:100790001197492F4A955E2F6F2FE89411274395A3
:1007A000203019F0C895802D01C080818823B9F0D0
:1007B0007C917723A1F0781739F40EF0042F13956C
:1007C000689411963196EBCF112321F0411BA11BA8
:1007D0001127B10BE894E52FF62F1196E0CF88236F
:1007E00011F0002708950895C895319600200895C6
:1007F000813618F08B3708F48F7D08950F920F9390
:10080000AF93BF938F939F938FB78F930024A7E8E5
:10081000B0E08091B9009091BA00891759F49CB169
:10082000A80FB01D9C938395823309F48827809389
:10083000B9000DC0082F0395023309F400270917EA
:100840009CB129F0A80FB01D9C930093B9008F9123
:100850008FBF9F918F91BF91AF910F910F9018957E
:10086000000F111F221F331F089500271127222771
:1008700033278D91882379F0F3DFF2DFF1DFF0DFAA
:10088000B7DF815408F4895F865F080F8827181F37
:10089000281F381FEECF089581918D938823E1F7AB
:1008A00008958FEF83959D919923E1F708956894BA
:1008B00001C0E894AF93BF938D9116F0919102C05F
:1008C00093DF902D891718F011F48823A9F7BF91B1
:1008D000AF91089541544D454C2072656164790093
:1008E00041004154450000004F4B000041545E0060
:1008F0003E2000002020202020202020202020201A
:100900002020202020202020200030440000202013
:1009100020200000454E53002020202020202020B1
:100920002020202020202020202020200000202007
:10093000205349454D454E5300004F20202020466E
:1009400046002020202020204D5033204F464600D6
:100950004F4646004D5033204F464600324400007B
:100960002D00324500002E00324600002F0033419A
:1009700000003A00334300003C00334500003E00D5
:10098000344100004A00344200004B003443000070
:100990004C00344400004D00344500004E00344605
:1009A00000004F00354100005A00364100006A0047
:1009B000364200006B00364300006C0036440000F5
:1009C0006D00364500006E00364600006F0037416E
:0409D00000007A00A9
:00000001FF
